:020000000B2DC6
:08000800FF00030E8312031335
:10001000A0000A0EA100040EA2008A110A120E2DE1
:10002000CE08031D1428080009300000FF3E031D00
:10003000152800000000CE0B14280800B708031D87
:1000400022280800F9300000000000000000000035
:1000500000000000000000000000000000000000A0
:10006000000000000000FF3E031D232800000000E8
:100070000000000000000000000000000000000080
:100080000000000000000000000000000000B70BAE
:1000900022280800FA30B7001E20FA30B7001E20D0
:1000A000FA30B7001E20FA30B7001E20B50B4A28E0
:1000B000080083120313AF08031D0800A701AA015B
:1000C000AC01AE013630831606048600363083124A
:1000D0000605B400163A031D72280330AF00013044
:1000E000A70083283408263A031D7B280330AF007D
:1000F0000130AA0083283408323A031D83280330D4
:10010000AF000130AC0002308316060486000230D6
:1001100083120605CF00D00102304F020319D00A26
:100120005008AE002E03031908000430AF00080089
:100130008316981683120C1E9A284F0899000800FF
:10014000D001D101D201FF30D300D401D5014F0A33
:10015000031DAC280130D4001816D508031DC32890
:100160008C1EB5280230D500AD28D408031DAD285B
:10017000CF08031DBE280130D500AD28D003D0081C
:100180000319CF03AD285508023A031DD328181DC3
:10019000CC281A08D200D328981CD1281812181677
:1001A000D3281A08D3005308D600080064308312FD
:1001B0000313CF00A0205608AD003003031DE5282F
:1001C0002D08B2000230B00008002D08B100013047
:1001D000AB0008005920AF0803195C292F08043A26
:1001E000031D00292908CF00D001CF0A0319D00A26
:1001F0000F304F05A9000130AF002D30B300552955
:100200002F08033A031D1429DF30831607058700E2
:10021000DF3083120705CF0020304F048700023003
:10022000AF009830B30055292F08023A031D4D291D
:100230000130AF00FE30831608058800FE308312BF
:100240000805CF0001304F048800FE3083160805F2
:100250008800FE308312080588002908CF00982006
:100260002703031D39291230CF0098200130A80040
:1002700055292A03031D42291C30CF009820013044
:10028000A80055292C03031D55290130B0001E304C
:10029000CF0098200130A8005529DF3083160705CC
:1002A0008700DF30831207058700B308031D5A2932
:1002B000AF015C293303B300A308031D6329A4081D
:1002C000031D63296A2901302302CF00031CA40304
:1002D0004F08A300A508031D7129A608031D712955
:1002E000080001302502CF00031CA6034F08A5001B
:1002F0000800C001C101C301C401C201421A0800C3
:100300000310C30DC40DBA0DBB0DC00DC10D3D08CA
:100310004102031D8D293C084002031C96293C081C
:10032000C0023D08031CC103C1024314C20A7E2956
:100330000808CD004D12CD124D13CD13CD10CD11A7
:100340004A0E0F39CE000F304E05CC004C184D161A
:10035000CC18CD164C194D17CC19CD17CB08031D51
:10036000CD144D0888000A30CE00102088150A30C0
:10037000CE00102088110F304A05CC000A30CE0084
:1003800010200808CD004D12CD124D13CD13CD1005
:10039000CD114C184D16CC18CD164C194D17CC1943
:1003A000CD17CB08031DCD144D0888000A30CE00B0
:1003B000102088150A30CE00102088110A30CE0097
:1003C00010200800B61FF1292D30CA001030CB00D4
:1003D00098213508003CBA00B6090318B60A3A0855
:1003E000B5003508B7003608B80027303602031DBF
:1003F000FB2910303502031C2F2AB61B2F2ABE0101
:100400003708BA003808BB00B81F0C2ABA09BB0964
:10041000BA0A0319BB0ABE0A1030BC002730BD005F
:1004200079214308B9003E1C172AB909B90A3908CD
:10043000303ECA001030CB0098213908003C031828
:100440002F2A10303702BA002730031C2830380218
:10045000BB003A08B7003B08B800B9031D2A0330B7
:100460003602031D352AE8303502031C6A2AB61B02
:100470006A2ABF013708BA003808BB00B81F462AED
:10048000BA09BB09BA0A0319BB0ABF0AE830BC00A3
:100490000330BD0079214308BE003F1C512ABE092C
:1004A000BE0A3E08B900303ECA001030CB00982189
:1004B0003908003C03186A2AE8303702BA000330D2
:1004C000031C04303802BB003A08B7003B08B800F0
:1004D000B903582A3608803ABA0080303A02031D20
:1004E000732A64303502031CA02ABF013708BA0002
:1004F0003808BB00B81F822ABA09BB09BA0A031917
:10050000BB0ABF0A6430BC00BD0179214308BE00AC
:100510003F1C8C2ABE09BE0A3E08B900303ECA0004
:100520001030CB0098213908003C0318A02A643011
:100530003702BA00031CB8033A08B700B903932A7C
:100540003608803ABA0080303A02031DA92A0A30E0
:100550003502031CD62ABF013708BA003808BB0091
:10056000B81FB82ABA09BB09BA0A0319BB0ABF0ADD
:100570000A30BC00BD0179214308BE003F1CC22ADD
:10058000BE09BE0A3E08B900303ECA001030CB009A
:1005900098213908003C0318D62A0A303702BA00DD
:1005A000031CB8033A08B700B903C92A3708303E1C
:1005B000CA001030CB0098210800013083120313C9
:1005C000CA00CB0198210230B7001E200230CA00B9
:1005D000CB0198210230B7001E200800C90148084D
:1005E0004902031808008313361883173508490792
:1005F0008400800803190800831336188317350810
:10060000490784000008CA001030CB009821C90AAD
:10061000EF2AB608031D0F2B8030B600112BC03017
:10062000B60035083607CA00CB0198210230B70062
:100630001E2008008316031308128812081388135B
:10064000881088110C308312B7001E203330CA0086
:10065000CB0198210230B7001E203230CA00CB01F6
:1006600098210230B7001E202C30CA00CB019821FF
:100670000230B7001E200630CA00CB01982102309C
:10068000B7001E200C30CA00CB0198210230B70001
:100690001E200130CA00CB0198210230B7001E2075
:1006A0000230CA00CB0198210230B7001E2008009A
:1006B000DF308316031307058700DF308312070539
:1006C0008700FB30831608058800FB30831208057D
:1006D00088001A23B501B60109232030BC00BF00F1
:1006E000C3002D30C1002E30BB003C30C0003E3076
:1006F000C2004330B7004730BE004C30C500553013
:10070000BD00C4006D30B900BA006F30B800C6013A
:100710000030C9003730B5004908B6000F30C800B6
:10072000EE22B5010130B60009232030BC00C00024
:10073000C3002D30C1003130BF003430C6003E3020
:10074000C2004230BD00C4005030BE00C500613060
:10075000B7006930BB007030B800B9007530BA001E
:10076000C7010030C9003730B5004908B600103065
:10077000C800EE220230B5004A20DD220730A90071
:10078000A801AB01AF01A301A401A501A601831635
:1007900081120116F03001058312B50006303504D0
:1007A000831681008B178B169030831298008B175D
:1007B00083168C1681138901FF3083128900FC3067
:1007C000831607058700FC3083120705B500033048
:1007D00035048700CB30831605058500CB308312A6
:1007E0000505B50034303504850008008312031375
:1007F0002B03031D412CAB012C30A5000130A600BA
:10080000B5010130B60009232030B900BC002D30FD
:10081000BB003C30BA004730B8005530B700BD01CE
:100820000030BE003730B5003E08B6000630C800C4
:10083000EE223208B500B601E2212E30B700B80131
:100840000030B9003730B5003908B6000130C800B3
:10085000EE223108B500B601E2212030B700B80021
:10086000B900BA00BB00BC00BD00BE00BF01003033
:10087000C0003730B5004008B6000830C800EE228E
:1008800008000130250226080318482C03194A2CB9
:10089000A61F0800B5010130B60009232030B700BB
:1008A000B800B900BA00BB00BC00BD00BE00BF006C
:1008B000C000C100C200C300C400C500C600C7011B
:1008C0000030C9003730B5004908B6001030C80004
:1008D000EE220800831203132803031DB42CA80181
:1008E0002C30A3000130A400B501B601092320304B
:1008F000B900BC002D30BA003E30BB004730B80014
:100900005530B700BD010030BE003730B5003E089D
:10091000B6000630C800EE222908B500B601E22173
:100920002E30B700B8010030B9003730B5003908B3
:10093000B6000130C800EE222703031DA42C12309C
:10094000B500B601E22108002A03031DAC2C1C30BF
:10095000B500B601E22108002C03031D08001E307B
:10096000B500B601E2210800013023022408031873
:10097000BB2C0319BD2CA41F0800B501B601092327
:100980002030B700B800B900BA00BB00BC00BD0001
:10099000BE00BF00C000C100C200C300C4010030DF
:1009A000C5003730B5004508B6000D30C800EE224E
:1009B00008000730831603139F000430980081302D
:1009C0009900831298019817C0308316810058232C
:1009D0006A24F6230D30B500B60109234130B70073
:1009E000B8010030B9003730B5003908B600013021
:1009F000C800EE222908B500B601E2212030B70078
:100A0000B8010030B9003730B5003908B600013000
:100A1000C800EE22E82C8A110A12D92C0B1D122DC7
:100A2000EA200B11831203138C1E182DD6208C1272
:100A3000220E8400210E8A00200E8300FF0E7F0EFE
:020A40000900AB
:02400E003A3F37
:00000001FF
